:1000000008308A000B2A0000FF00030E8301A100C4
:100010000A08A0008A010408A2007708A300780853
:10002000A4007908A5007A08A6007B08A70083131E
:1000300083120B1E1D288B1842288C308400801ED2
:1000400023288C1A45288C308400001C29280C1881
:1000500048288C308400801C2F288C184B282208BC
:1000600084002308F7002408F8002508F900260872
:10007000FA002708FB0020088A00210E8300FF0EEB
:100080007F0E09008A110A129A298A110A12802801
:100090008A110A1268298A110A1278290A108A100C
:1000A0000A11820730342E34363400340A108A1094
:1000B0000A1182075734443454340D340A3400345E
:1000C0000A108A100A11820743344F344D344D34DC
:1000D00041344E34443420344534523452344F3455
:1000E00052340D340A34003464008C1E742818080D
:1000F000EE001A08F800EE1C7F28181218160034BB
:10010000A0307107840083130317EA010408E90093
:100110006A10831B6A140313742003176908840090
:1001200083136A18831778088000A0307107840051
:1001300083130008243C031DA6280130F200F101BE
:10014000243083160313A00083120317F208031947
:1001500063297108043C031DC52804307102703EF8
:10016000F800FA010318FA0A7808E8007A08E900AA
:10017000A0307107840083130008EA006808840037
:100180008313691883176A0880000130F10771082A
:10019000063C03186329F201F10101300313EF005B
:1001A000831621082F3C0318D9282108393C03184D
:1001B000E9282108403C0318E1282108463C03189F
:1001C000E9282108603C031816292108663C031C15
:1001D000162922082F3C0318F1282208393C03185D
:1001E00001292208403C0318F9282208463C03183C
:1001F00001292208603C031816292208663C031CCA
:1002000016292208393C031807290930A2070F30A4
:10021000A2052108393C03180F290930A1070F3026
:10022000A1050310210D2204F30019298312EC16F5
:10023000831625082F3C031821292508393C03186B
:1002400031292508403C031829292508463C031874
:1002500031292508603C03185E292508663C031CEB
:100260005E2926082F3C031839292608393C031833
:1002700049292608403C031841292608463C031812
:1002800049292608603C03185E292608663C031CA1
:100290005E292608393C03184F290930A6070F307C
:1002A000A6052508393C031857290930A5070F3042
:1002B000A5050310250D2604F400612983126C178F
:1002C00083168312031703138C128A110A122F2824
:1002D000D80B74290130D0070318D10A0319D20AA8
:1002E0000319D30A0F30D8000C108A110A122F28D4
:1002F000D90B84290130D4070318D50A0319D60A6B
:100300000319D70A6230D9008C108A110A122F28DB
:1003100083160C1083125308DD005208DC005108CC
:10032000DB005008DA0058080F3CE20083160C147A
:10033000831200346C1CA729EC18A7296C1AA72972
:1003400088210616831606128312EC14AE296C1847
:10035000AE296C19AE296C1AAE296C158B108A1156
:100360000A122F288C1EB6297420B22983168612F1
:10037000831286120034F515750883168700003045
:100380008312871D0130F700770D8316C900C90D50
:10039000C90DF830C905751575088700003083123E
:1003A000071D0130F700F70DF70DFC30F705770852
:1003B00083164904CB00F5147508870000308312BA
:1003C000871C0130F7000310F70D770883164B04E4
:1003D000CD0075147508870000308312071C0130AA
:1003E00083164D048312ED00B221EF0183168C16A3
:1003F000C03083128B048A150A128C2A7C08840070
:1004000083137D18831703173A088000840A80013C
:10041000FC0A0319FD0A031300340317B91B222A2F
:100420000F30F700380EF7050A30770203181B2A41
:100430003030F7071D2A3908F7077708BA00031389
:10044000FE2103170F30B8050A30380203182A2A94
:1004500030302C2AB9133908B8073808BA0003130A
:10046000FE21003403173908BE003808BD003E08DD
:10047000FA003D08840083137A1883178008031953
:10048000452ABD0A0319BE0A372A3B08FA003A0872
:10049000840083137A18831780080319692A3C089B
:1004A000003C0318692A3A08840083133B18831719
:1004B0000008C1003D08840083133E1883174108DB
:1004C0008000BD0A0319BE0ABA0A0319BB0ABC039D
:1004D000452A3D08840083133E188317800138089D
:1004E000F8003908F90003130034831686128312CA
:1004F0008616003475220317BA01B9013A08013C87
:10050000031CA22A031D882A3908903C031CA22A36
:10051000F51775088316031387008312871B952A26
:100520000317BA01B9019B2A031364001030F700C6
:10053000F70B982A0317B808031D6400B90A0319BA
:10054000BA0A7E2A0313B22100340C1EA52A03170F
:100550004108031399008A110A12E42A40308400EA
:10056000831700080319C52A0130F800BF30F700CF
:100570006400F70BB82AF80BB62A4A30F700F70BDD
:10058000BF2A00006400800BB42A003403173F1018
:10059000031375220317BC013C08043C031CFE2A0C
:1005A00003136E130317BD0139083D020318EA2A2D
:1005B0003B08FA003A08840083133B1883170008AD
:1005C000C000C1000313A52A0317BA0A0319BB0A06
:1005D000BD0AD42A03136E1BF62A4F080317C00066
:1005E0000313AE2203173F14FE2A03134F08031709
:1005F000C0000313AE220317BC0ACC2A0313B22196
:10060000003003173F180130F800031300340130A5
:10061000FD001030FC003F300317BA000313FE2129
:100620006D080317B8005730B90003130D222030AE
:100630000317BA000313FE2101300317B90010306D
:10064000B80083160313490883120317BB008316EF
:100650000313480883120317BA001030BC000313B9
:10066000322279088316C9007808C800CA014A08EE
:100670004807840083134918831780080319422B05
:10068000CA0A372B83120317B80103137A226D08A5
:100690000317B800831603134A0883120317B9001F
:1006A00083160313490883120317BB008316031331
:1006B000480883120317BA000313C622F808031D63
:1006C000672B0A300317C0000313AE22472B0034F8
:1006D0008316C9080319742B8312EF080319722BB0
:1006E0008316742B682B83168312EF08031D7C2B53
:1006F0000030F8008C2B8C2B6D087302031D872BA8
:10070000EC1A872BEF010130F8008C2B8C2BEC12AC
:10071000EF010030F8008C2B8A150A12FA2A831692
:100720004908FA004808840083137A1883170008E0
:10073000CC004B08FA004A08840083137A18831708
:1007400000084C02031DBB2B4908FA00480884002E
:1007500083137A1883178008031DB12B0030F8002B
:10076000D42B4908FA004808C80A0319C90ACA0A5A
:100770000319CB0A902B4908FA0048088400831318
:10078000491883170008CC004B08FA004A08840077
:1007900083134B18831700084C020318D22BFF3029
:1007A000FA00D32B0130F8008312003483160C10AA
:1007B0008312D301D201D101D0010F30D8008316AA
:1007C0000C148C108312D701D601D501D4016230EC
:1007D000D90083168C148312061583160611831212
:1007E0000712751275088316870083128716F51293
:1007F00075088316870083126C148A150A120E2B53
:1008000020308316D400D001D101D201D3014B088E
:10081000FA004A08F9004908F8004808F7000310F0
:10082000771C202C4C08D0074D0803184D0FD1071A
:100830004E0803184E0FD2074F0803184F0FD30767
:10084000D30CD20CD10CD00CFA0CF90CF80CF70C20
:10085000D40B0F2C831200348E30F70083164D0812
:10086000F8004C08F900FA01F808031D412C79083A
:10087000F800F9010830F702F808031D412CF701D0
:10088000492C0310F81B482CF90DF80DF703412CE7
:10089000F8138312003483164C080319BC2CD400BF
:1008A00050080319BC2CD40703185D2C7F30D402E8
:1008B000031CBC2C0319BC2C612C8130D4070318F9
:1008C000BC2C5408F700F801F901FA014D08D800D2
:1008D000D8174E08D7004F08D6001830D400D501DD
:1008E000561C8A2C5308FA07031C7C2CF90A031D9A
:1008F0007C2CF80A0319D5175208F907031C832C1E
:10090000F80A0319D5175108CE00CE174E08F8077C
:100910000318D517D50DF80CF90CFA0CD80CD70C18
:10092000D60C0310D40B6F2C0130F7070318BC2C26
:10093000F81BA12CD80DFA0DF90DF80DF7030319CA
:10094000BC2CD81FB22CFA0A031DB22CF90A031DC5
:10095000B22CF80A031DB22CF80CF90CFA0CF70AA9
:100960000319BC2C4D08D5005108D506D51FBA2C4B
:10097000F817C02CF813C02CF701F801F901FA019F
:1009800083120034B630F700FA01F901F80183163A
:100990005008510452045304031DD02CF701DD2CE0
:1009A0000310F81BDC2CD00DD10DD20DD30DFA0D98
:1009B000F90DF80DF70BD02CF813831200348030AA
:1009C000831CE52C8316D50683128316DA01DB011E
:1009D0005108D9005508D90650080319D32DD8005D
:1009E000F70054080319DC2DD8020319782D031CD5
:1009F000362D5508DE00DE175608DD005708DC00EE
:100A0000DB010310DE0CDD0CDC0CDB0CD80B002D45
:100A1000D91F0D2D5A14F02D5A1058105A16D330D4
:100A200084008313052E5A12D91B202D581C2B2D00
:100A3000DE0CDD0CDC0CDB0CF70A0319EB2D2B2D87
:100A4000DE1B2E2D0310DB0DDC0DDD0DDE0DF7039F
:100A50000319EB2D202D5A17982D5A135108D90040
:100A6000D91F342DDE17E42DDE13E42D5408D800F1
:100A7000F7005008D8025108DE00DE175208DD00EA
:100A80005308DC00DB010310DE0CDD0CDC0CDB0C9E
:100A9000D80B422DD91F4F2DDA14F02DDA10581033
:100AA000DA16D73084008313052EDA12D91B622D93
:100AB000581C6D2DDE0CDD0CDC0CDB0CF70A031969
:100AC000EB2D6D2DDE1B702D0310DB0DDC0DDD0D10
:100AD000DE0DF7030319EB2D622DDA17982DDA13CB
:100AE0005508D900D91F762DDE17E42DDE13E42D2D
:100AF0005508DE00DE175608DD005708DC00D91F58
:100B0000852DDE135A15F02D5A11DB015810D33004
:100B100084008313052ED91BAE2D5108D900581C13
:100B2000982DDE0CDD0CDC0CDB0CF70A0319EB2D29
:100B3000DB1FA92DDC0A031DA92DDD0A031DA92D2C
:100B4000DE0A031DA92DDE0CDD0CDC0CF70A0319EF
:100B5000EB2D5A1B2D2DDA1B6F2DCD2D8030DE068F
:100B6000DE1FB62DF02D5508D900C32D5108D90030
:100B7000DE08031DC32DDD08031DC32DDC08031D86
:100B8000C32DF701E42DDE1BCD2D0310DB0DDC0D95
:100B9000DD0DDE0DF70BC32DEB2DD91FD12DDE178B
:100BA000E42DDE13E42D5408F7005508DE00560846
:100BB000DD005708DC00E42D5008F7005108DE0086
:100BC0005208DD005308DC005E08F8005D08F900FB
:100BD0005C08FA00232EF701F801F901FA01232E2F
:100BE000DB01DC09DD09DE09DB09DB0A031DFE2D63
:100BF000DC0A031DFE2DDD0A0319DE0A5A180C2D2E
:100C0000DA184E2D5A19842DB32D0008DC07031C69
:100C10000F2EDD0A031D0F2EDE0A0319581484035C
:100C20000008DD07031C172EDE0A0319581484037D
:100C30000008801F803ADE07031858145A1A132D33
:100C4000DA1A552D8B2D8312003483165008B63CCA
:100C5000D000FA015108D400D1170310D10CD20CE6
:100C6000D30CFA0CF90CF80CF70CD00B2D2ED41F6A
:100C7000442EF709F809F909FA09F70A0319F80ADD
:100C80000319F90A0319FA0A83120034F701F8016B
:100C9000F901FA018316DC01DD01DE01DF015B08E9
:100CA0005A04590458040319852E2030E00003101B
:100CB000D40DD50DD60DD70DDC0DDD0DDE0DDF0D00
:100CC0005B085F02031D6E2E5A085E02031D6E2E26
:100CD00059085D02031D6E2E58085C02031C7F2E0E
:100CE0005808DC025908031C590FDD025A08031C7E
:100CF0005A0FDE025B08031C5B0FDF020314F70DC3
:100D0000F80DF90DFA0DE00B572EDC30840083133B
:100D10008312003404088316CC00CB1F9C2ECC0316
:100D2000CC16C809C909CA09CB09C80A0319C90AD6
:100D30000319CA0A0319CB0A3B30D3009A30D200F8
:100D4000CA30D100D0010A30CE004B08D7004A0883
:100D5000D6004908D5004808D4005308DB005208E3
:100D6000DA005108D9005008D8008312462600083E
:100D70008316C800840A0008C900840A0008CA0053
:100D8000840A0008CB00F708031DD92E4E08013A4B
:100D90000319D92E4C080319DB2E0F394E02031903
:100DA000D32E0318032FCC1B032F4C1BDB2E20301C
:100DB000FB2E2030CC05CC1EEA2ECC127708CC00BE
:100DC0002D3083120317BA000313FE2183164C083B
:100DD000F700CC013030CC1EFB2ECC127708CC00B3
:100DE0002D3083120317BA000313FE2183164C081B
:100DF000F700CC013030F707770883120317BA00E9
:100E00000313FE2183165308D7005208D600510859
:100E1000D5005008D400DB01DA01D9010A30D8002E
:100E2000831246267A088316D3007908D200780800
:100E3000D1007708D000CE0BA52E83120034861483
:100E4000831686100130FD001030FC002A3083121A
:100E50000317BA000313FE216D080317B8005730BB
:100E6000B90003130D2201300317B9001030B80088
:100E700083160313490883120317BB008316031359
:100E8000480883120317BA001030BC000313322243
:100E900079088316C9007808C800CA014A084807BB
:100EA000840083134918831780080319592FCA0A2D
:100EB0004E2F83120317B80103137A226D0803170C
:100EC000B800831603134A0883120317B900831668
:100ED0000313490883120317BB0083160313480842
:100EE00083120317BA000313C622F808031D7E2FCE
:100EF0000A300317C0000313AE225E2F861083163C
:100F000086108312003400306C180130F700770D22
:100F10008316C900C90DC90DF830C9050030831208
:100F2000EC1B0130F700F70DF70DFC30F7057708E3
:100F300083164904CB0000308312EC180130F7000F
:100F40000310F70D770883164B04CD000030831291
:100F50006C19013083164D04F600FD013B30FC0096
:100F6000760883120317B8005730B90003130D2217
:100F70000D300317BA000313FE210A300317BA001D
:100F80000313FE218316C9013B30C80083121F27BB
:100F90008A150A12302BFD013B30FC008316C80174
:100FA000480883124E2000380319E02F8316C80A20
:100FB00083120317BA000313FE218316D02F831266
:100FC0000D300317BA000313FE210A300317BA00CD
:100FD0000313FE218316C9013B30C80083121F276B
:0E0FE0008A150A12422BF32F8A150A12642B6F
:101000006C1C8428EC1C84285D088316CB0083129A
:101010005C088316CA0083125B088316C90083121A
:101020005A088316C800CF01CE010330CD00E83046
:10103000CC008A11831200248A157A088316CB000B
:101040007908CA007808C9007708C800CD01831262
:1010500062088316CC008A1183122C248A157A0820
:101060008316CF007908CE007808CD007708CC0031
:101070004D30D3005530D2000530D1008530D0003E
:101080008A1183124B248A1577088316CC007808BE
:10109000CD007908CE007A08CF004B08D3004A086B
:1010A000D2004908D1004808D0008A118312C22416
:1010B0008A1583107A088316D3007908D20078083D
:1010C000D1007708D0004F08D7004E08D6004D0851
:1010D000D5004C08D4008A118312DF248A157A08BF
:1010E0008316D3007908D2007808D1007708D000A1
:1010F0008A11831225268A157A08E7007908E60006
:101100007808E5007708E400FD013B30FC00413041
:10111000840067088316CB00831266088316CA0012
:10112000831265088316C900831264088316C800F9
:101130008A1183128A268A150D300317BA008A1184
:101140000313FE218A150A300317BA008A1103130C
:10115000FE218A158316C9013B30C8008A1183120B
:101160001F278A158A150A121F2BFD013B30FC0030
:10117000413084006B088316CB0083126A08831603
:10118000CA00831269088316C9008312680883168F
:10119000C8008A1183128A268A150D300317BA00F7
:1011A0008A110313FE218A150A300317BA008A1127
:1011B0000313FE218A158316C9013B30C8008A112A
:1011C00083121F278A158A150A12532B8316480883
:1011D0000319AC29D4004C080319AC29D402031C10
:1011E000F6287F30D4070318AC29FC288130D402BC
:1011F000031CAC290319AC295408F700F801F901C4
:10120000FA01D3014908D200D2174A08D1004B088D
:10121000D0001930D4004F08D00203181F29013024
:10122000D10203181F29D20203181F29D302031861
:101230001F29D30AD20AD10A4F08D00751294E08D4
:10124000D10203183A290130D20203183A29D302F5
:1012500003183A29D30AD20A4E08D1074F08D007FB
:10126000031C5129D10A031D5129D20A031D5129FA
:10127000D30A51294D088038D20203185029013071
:10128000D30203185029D30A4D088038D2074E08DC
:10129000D107031C2E29D20A031D2E29D30A2E2979
:1012A0007A14D40B54295F290310D00DD10DD20D1F
:1012B000D30D0310FA0DF90DF80DD50D0B29551CA2
:1012C00067290310F80CF90CFA0CD50C6A29F703FE
:1012D0000319AC29D51B93290310D00DD10DD20DC4
:1012E000D30D4F08D00203187F290130D102031813
:1012F0007F29D20203187F29D302031CA2294E089A
:10130000D10203188A290130D20203188A29D30294
:10131000031CA2294D088038D202031893290130FA
:10132000D302031CA229FA0A031DA229F90A031DEC
:10133000A229F80A031DA229F70A0319AC29F80CFF
:10134000F90CFA0C4908D4004D08D406D41FAA2978
:10135000F817B029F813B029F701F801F901FA01DB
:1013600083128A150A12C62B83164908D0004D082D
:10137000D006D01FC02903110310C91B0314F32981
:101380004908D0004C08D1004808D1020319CE29E1
:10139000D01FF3290308013A8300F3294D08D10037
:1013A0004908D1020319DA29D01FF3290308013AA9
:1013B0008300F3294E08D1004A08D1020319E62917
:1013C000D01FF3290308013A8300F3294F08D10005
:1013D0004B08D1020319F229D01FF3290308013A5F
:1013E0008300F329031083128A150A12F82B83163F
:1013F0008C1083125708E1005608E0005508DF0002
:101400005408DE005908623CE30083168C148312F2
:101410008A150A12FD2B840183131F3083051930AE
:1014200083169900A6309800903083129800831696
:101430001F149F141F159F1107309C008312A901D0
:10144000AA014630AF00B0015130B100B2015330B3
:10145000B300B4015630B500B6014130B700B80151
:101460005230B900BA010330CF00D001D101D2010E
:10147000D301D401D501D601D701D801D901DA01B0
:10148000DB01DC01DD01DE01DF01E001E101E20160
:10149000E301E401E501E601E701E801E901EA0110
:1014A000EB016C10EC106C11EC116C12EC126C1363
:1014B000EC13ED01EE01F201FF30F300F401F50051
:1014C000FC01FD01F601FE018316BE01BF014310C0
:1014D00001130F308312D8006230D9000C30F700AE
:1014E000073081018130840083130008F039073808
:1014F000800064000008F739F719F039770480009C
:10150000853090004830F80005389200FF3083168F
:1015100092008A118312BB298A150B1683160C14AC
:101520008C148312071675127508831687008312B0
:101530008712F512750883168700831286108316AA
:101540008610831206118316061183120612831663
:1015500006121F1383121F179F1783169F138312E0
:101560001F1483161F109F141F159F150030F800BD
:1015700083121F08C73978049F0003081839F70041
:1015800083160E08033977040E148E148315031680
:101590000B3A83120319D02A133A0319F12AF22ABB
:1015A000FD013B30FC008316C80148088A118312F4
:1015B00056208A158316C80AF70083120317BA004B
:1015C0008A110313FE218A15053083164802031D74
:1015D000D52AC9013B30C8008A11831207238A1516
:1015E000F22AF22A64006D088316C800C9018A1124
:1015F0008312682B8A15F8080319862B8316C901F4
:101600007030C800CB012F30CA008A1183128F239B
:101610008A15F808031D102B8A11D62B8A15862BE4
:101620008316C9017030C800CB013130CA008A115D
:1016300083128F238A15F808031D202B0028862B80
:101640008316C9017030C800CB013330CA008A113B
:1016500083128F238A15F808031D322B8A11832FDA
:101660008A15862B8316C9017030C800CB0135302E
:10167000CA008A1183128F238A15F808031D442B90
:101680008A11CB2F8A15862B8316C9017030C800AA
:10169000CB013730CA008A1183128F238A15F808CC
:1016A000031D542BB528862B8316C9017030C80042
:1016B000CB013930CA008A1183128F238A15F808AA
:1016C000031D662B8A11F32F8A15862BFD013B30F3
:1016D000FC008316C80148088A11831260208A150D
:1016E0008316C80AF70083120317BA008A1103137E
:1016F000FE218A150F3083164802031D6B2BC9018A
:101700003B30C8008A11831207238A156C1C9D2B5D
:10171000EC189D2B6C1A9D2B8A1188218A15DD08E7
:10172000031D9C2BDC08031D9C2BDB08031D9C2B3D
:101730005A081D3C03189D2B6C166C1C7F2CEC1951
:101740007F2C6C1A7F2C1F151F19A42B1E088316C3
:10175000CD01CC008A1183122C248A157A088316B5
:10176000C7007908C6007808C5007708C400470894
:10177000CB004608CA004508C9004408C800CF018C
:10178000CE01CD018730CC008312E628770883167E
:10179000C8007808C9007908CA007A08CB00CF00D1
:1017A0004A08CE004908CD004808CC00D301D20138
:1017B0002030D1008130D0008A1183124B248A1549
:1017C0007A088316C7007908C6007808C50077082C
:1017D000C400CB01CA01C9018030C8004708CF004E
:1017E0004608CE004508CD004408CC008312B42939
:1017F0000318FC2B031D7F2CF72961088316CB00EF
:10180000831260088316CA0083125F088316C9001A
:1018100083125E088316C800CF01CE010330CD00CD
:10182000E830CC008A11831200248A157A088316C6
:10183000CB007908CA007808C9007708C800CD0134
:10184000831263088316CC008A1183122C248A1514
:101850007A088316CF007908CE007808CD00770883
:10186000CC009630D3004330D2002330D1008230F8
:10187000D0008A1183124B248A1577088316CC0076
:101880007808CD007908CE007A08CF004B08D30045
:101890004A08D2004908D1004808D0008A118312B2
:1018A000C2248A1583107A088316D3007908D200DF
:1018B0007808D1007708D0004F08D7004E08D6002E
:1018C0004D08D5004C08D4008A118312DF248A15F4
:1018D0007A088316D3007908D2007808D1007708F7
:1018E000D0008A11831225268A157A08EB00790820
:1018F000EA007808E9007708E800EC15EC176C1CA2
:0E190000852CEC18852C6C1E852CF22A6300B9
:02400E00753FFC
:00000001FF
